:030000000219FDE5
:03000B000200AA46
:03002B0002015778
:03005B000202E3BB
:030073000202D0B6
:1000800002030406080C10182030406080040608A3
:100090000C10182030406080A0C00003070F1F0D17
:1000A0000D0403060D0502030202C2AFC0D0C0E07A
:1000B000206214E5256009E473E525F4F58AD2622F
:1000C000D0E0D0D0D2AF3285268AC262E526F46075
:1000D0002AD0E0D0D0C295C294C293D2AF32C2959A
:1000E000C294C293206F0D20650A7405D5E0FDE52A
:1000F0007BF45290D0E0D0D0D2AF32758A00C28D5E
:10010000D26201F401B9306805206502D29501B9C7
:10011000306805206502D29401B930680520650277
:10012000D29301B9D29230680A2065077403D5E0F2
:10013000FDD29501B9D29130680A2065077403D5C4
:10014000E0FDD29401B9D29030680A2065077403AB
:10015000D5E0FDD29301B9C2AFC2AD53E6EFC0D036
:10016000C0E0D2D3D2AFC2CEE52A600720744915D1
:100170002A21B87800790020742EE580307E01F4C1
:1001800030E70278FF53DACF207E0343DA20307E57
:100190000343DA10C2D8C271E580307E01F430E743
:1001A0000279FFC3E89970CB306103752A4020744F
:1001B00003752A40885CD27020740DE52B6004150D
:1001C0002B21C843DA01C2D820700221DBA85C20B1
:1001D0006102C27020740221D988227882B6040399
:1001E00085222420CF0AD0E0D0D043E610D2AD3211
:1001F000C2CF053A7802E52A6005307402152AC399
:10020000E55C94014005755F00411C7560007569EF
:1002100000E55F2401F55F5003755FFF7982B70247
:100220000D306E1DC3E52294324016854C22798232
:10023000B7030E306E0BC3E52294324004798E87EB
:1002400022C3E5239522600840041523415005236D
:10025000D8CA0569E56970021569D56A69756A01C8
:100260007808E56B60497805C3E569956B4057C32D
:10027000E569956C50087801756A0302028AC3E546
:1002800069956D50057801756A01C3E56295244052
:100290001E7982B7040241BB206E14852462E56991
:1002A000046003856B69756A0175233C0202C6E52B
:1002B000622850057562FF41BBF562E56204700675
:1002C0007560FF7569FFD0E0D0D043E610D2AD3243
:1002D000C2AF53E67F7592FA7593FFC260759104C1
:1002E000D2AF32C2AF53E6EFC2ADC0D0C0E0C0F073
:1002F000D2D3D2AFA8FBA9FCC2D8307102614A5355
:10030000DACF207E0343DA10307E0343DA20D27145
:10031000E580307E01F420E702612188278928A149
:100320002F53DACF207E0343DA20307E0343DA10E6
:10033000C2D8C271307402A11B7800E580307E0102
:10034000F430E702A11B885CA10353DACF207E03BF
:1003500043DA20307E0343DA10C271206102812328
:1003600053DACF207E0343DA10307E0343DA20C213
:10037000D8D27188578958C3E89555F8E99556F948
:100380007B007E087A00C3E8948CE99400500575E0
:100390005B008115882178A2E6A8216055C3E89406
:1003A000C8E994005008E4D2E4FB7A0A61F0C3E89B
:1003B0009468E994015008E4D2E3FB7A0F61F0C33A
:1003C000E894D0E994025008E4D2E2FB7A1E61F08E
:1003D000C3E894A0E994055008E4D2E1FB7A3C61BB
:1003E000F0C3E89498E994085008E4D2E0FB7A78E6
:1003F0007E00C3E89559FCE9955AFD30E70AECF414
:100400002401FCEDF43400FD755B00C3EC9AED9E15
:100410005003755B018859895A8557558558567818
:1004200002A103C3E89527F8E99528F9307C0281F9
:10043000E7307B0281E7307A0281E0207502814655
:10044000E9FDE8FC8165E9C313F9E813F8307902A6
:1004500081E0E9C313F9E813F830780281E0E9C3D9
:1004600013FDE813FC20612CC3EC941CED940240B6
:0E04700002817CED701EC3EC94C85018052963
:10047E00E52970021529C3E529940A5002A11B75BE
:10048E005C00D270A11BE529600215297400207F43
:10049E00037896E624FAFEE43400FFC3EC9EFCEDEE
:1004AE009FFD50067800790081E7C3EC94FFED9430
:1004BE0000400678FF790081E7EC8572F0A4C5F064
:1004CE00A2F733F87900400302050378FF790002A2
:1004DE000503E9C313F9E813F8307C0EE9600278DE
:1004EE00FFC3E81338F8E43400F9C3E894FFE99445
:1004FE0000400278FF885CD270206102A11B741F3D
:10050E00F4552F4BF52FC274EB7002D274752A403E
:10051E00307403752A0A306102A12F20740353DA56
:10052E00FE207403752B20D0F0D0E0D0D0D2AD4396
:10053E00E61032790102055F790302055F790A023E
:10054E00055F791E02055F796402055F79C80205B1
:10055E005F7817E4D5E0FDD8FAD9F6227A147B78C5
:10056E000205867A107B8C0205867A0D7BB4020515
:10057E00867A0B7BC8020586E573D5E001227902E7
:10058E00E4D291D5E0FDD294D5E0FDC294D5E0FD44
:10059E00C291D5E0FDE920E002D29530E002D2937F
:1005AE00E573D5E0FDE920E002C29530E002C2938A
:1005BE007496D5E0FDD9C9EAF8D5E0FDD8FBDBB8D5
:1005CE00D29122C37C007D0075F00005F0EA33FA6B
:1005DE00EB33FB50F6EB13FBEA13FAC3E9FFE8FE2D
:1005EE00E89AF8E99BF95004EFF9EEF8B3EC33FC16
:1005FE00ED33FDD5F0DFEDF9ECF822E889F08A2035
:10060E00D2D4F8A9F07B0030F70B7BFFF42401F86D
:10061E00E9F43400F9E88520F0A4ADF0F8E985207E
:10062E00F0A4AFF0FEED2EF974003FFA7C04C3EA9D
:10063E0013FAE913F9E813F8DCF48BF030F70AE853
:10064E00F42401F8E9F43400F9E889F0C2D4F8A9E9
:10065E00F0227882B604030206FFC3E55C941940CB
:10066E001EE52D54067018206E3678057994E71421
:10067E006007780A1460027812C3E54198401F3073
:10068E006E098564627569FF756A01852224E4F539
:10069E0044F545F546F547F548C26E0206FFD26EA3
:1006AE007994E7147013E523F43333F913F8E9540E
:1006BE000104F9E854FE0206F3E714147014E5235E
:1006CE00F4333333F913F8E9540304F9E854FC0214
:1006DE0006FBE523F433333333F913F8E9540704F7
:1006EE0004F9E854F8C39440F8E99400F988448971
:1006FE004522C3E54113F9E54013F8C3E54498F8E4
:10070E00E54599F9500CC3E89480E994FF40160230
:10071E000737C3E8947FE994005003020737787FC8
:10072E007900020737788079FF8849894A22E5499E
:10073E002546F8E54A3547F9854A20E4300701F4A5
:10074E003548FA30E709C3EA94F04015020775C33D
:10075E00EA940F500302077578FF79FF7A0F0207AC
:10076E0075780079007AF0C3E5249561500AC37458
:10077E00019524500B020793E54A20E70E020793DA
:10078E00E54A30E706884689478A482278A5E6FA80
:10079E00C3E54933F8E54A33F9D109E930E70BC32C
:1007AE00E89480E994FF4013E1CDC3E8947FE99487
:1007BE00005002E1CD787F7900E1CD788079FFE8B5
:1007CE0020E715C3E52398F84009C3E894014003D8
:1007DE000207F478010207F4E8F424012523F84017
:1007EE00030207F478FF884B2278A6E6FAA847A9F9
:1007FE0048120609E930E70CC3E89401E994FF407A
:10080E0016020829C3E894FFE99400500302082950
:10081E0078FF7900020829780179FFE920E715C3EE
:10082E00E54B98F84009C3E894014003020850785C
:10083E0001020850E8F42401254BF8400302085049
:10084E0078FF88242278FF20692879A1E76023E5C4
:10085E0041601F74FF8541F0848539F0306A03755D
:0E086E00F005A4F8C5F0600278FFC3E89564B9
:10087C005002A864886322C3E5409440E54194018A
:10088C00E5635003140194046002F563227883E657
:10089C00F520120F1475E89012054175E89030EDB3
:1008AC00FDA8BDA9BE120FBA756E55756F00C37445
:1008BC000013FD7455606613FC74552CFC74003DDC
:1008CC00FDECFAEDFBC3E89AE99B4014E56E245568
:1008DC00F56EE56F3400F56FEA2CFAEB3DFB80E525
:1008EC00AE6EAF6FC3E56F13F9E56E13F8C3E91382
:1008FC00F9E813F87A03C3E913F9E813F8DAF7AA5D
:10090C00201A7009756E00756F000209291AEA60C9
:10091C0008EE28FEEF39FFDAF88E6E8F6F2275E83D
:10092C0090227883E6FF30EDF9A8BDA9BE0570C30F
:10093C00E57094084052757000E9FA79A0E76044BC
:10094C00EA7007E571601B020962C3E895716010DB
:10095C00E5715006600C1402096E0460F902096E10
:10096C00E571F571C3946D401B7561C0C39404406F
:10097C0013756180C39404400B756140C3940440AB
:10098C000375610075BB0622EFC39401601F74559B
:10099C00601BC3E894FFE994035012C3E8956EE919
:1009AC00956F5009E561600C15610209C0E561F4B1
:1009BC0060020561A861C3E524985002A824C3E82D
:1009CC009562400AA862E562F4600385626188253D
:1009DC008826E570B4070375BB1022743279A7879B
:1009EC00F0A4C5F0A2F733F8C3E895614002A86102
:1009FC0088228824882588268864227540007541C1
:100A0C00F022C2AF75C820A8CCA9CDAA3A30CF012C
:100A1C000A75C824D2AFAB3BAC3C883B893CC3E8DD
:100A2C009BF8E99C206908F9306602611D4177AD9D
:100A3C003D8A3DF9EA9DFA600478FF79FFAE3EAF3E
:100A4C003F8B3E8C3FA83BA93CC3E89EF8E99FF93D
:100A5C00C3E54113FBE54013FAE82AF540E93BF501
:100A6C004150067540FF7541FF41C4AA40AB41ACF3
:100A7C0040AD417E047F02C3EB9404400D1E1FC3A6
:100A8C00EB94084005206A021E1FC3ED13FDEC1306
:100A9C00FCDEF7C3EA9CFAEB9DFBEF6009C3E9139C
:100AAC00F9E813F8DFF7EA28FAEB39FB8A408B41B7
:100ABC0050067BFF8B408B41C3EB94025002D266F5
:100ACC003069047F0341EF7892E6FFC3E5379482E7
:100ADC0040110FC3E53794A040010FC3EF940640BB
:100AEC00027F057E02E541C4540FF9E541C454F080
:100AFC00F8E540C4540F28F8C3E89EFAE99400FBCB
:100B0C004009C3EA9402EB940050047A02E4FB61BE
:100B1C0069AA40AB41EBC4FEEAC4540F4EFCC3EAD5
:100B2C009CFAEB9400FBC3E813C313F8EA28FAEB26
:100B3C003400FB8A408B41C3EB94024002C26678BE
:100B4C0002EBC4FE7B00EAC4540F4EFAC3EA98FAD7
:100B5C004005C3940250027A027892E6FF3060029C
:100B6C006169855192855293D26043E680C3E49AC1
:100B7C00F8E49BF930660261F5E8FAE9FBD3E91376
:100B8C00FDE813FC88518952C3EF94036038EF20C1
:100B9C00E00DE82CF8E93DF9ECFAEDFB020BBEE8B0
:100BAC0028F8E939F9C3E82402F8E93400F97AFEA7
:100BBC007BFFC3EF9403400E8A538B54884D894EB0
:100BCC008C4F8D508129885389548A4D8B4E8C4F74
:100BDC008D503069127553F07554FF754FF0755088
:100BEC00FF7551F07552FF8129E8FAD3E813FC88A0
:100BFC0051C3EF94036020EF20E007E82CF8ECFAE7
:100C0C008115E8282402F87AFEC3EF940340088A81
:100C1C0053884D8C4F812988538A4D8C4FE568C37E
:100C2C00335002646BF5683060028133753402D244
:100C3C006043E680E52D54066034A840A941C3E921
:100C4C0013F9E813F8C3E913F9E813F8306904E968
:100C5C002440F9C2AF53E67F759100C3E498F59434
:0F0C6C00E499F595759104D26043E680D2AF22EA
:100C7B00D264754300752000306C03752040020C64
:100C8B009AD264754300752040306C037520007850
:100C9B00017901206620E52D54066002C2647914A7
:100CAB00E541C313700104F8C39414400278143067
:100CBB006904781B791B206010E543600C306903D5
:100CCB00D53404D26DA144913B0543E59B5440B50B
:100CDB002002A12E30690908C3E89940011881C18F
:100CEB0020640A08C3E8994002819A81C1C264C298
:100CFB00AF53E67F7591003066127594007595F8C9
:100D0B00759104D26043E680D2AF819AE5417EFFB4
:100D1B00C3334005C3334001FEC3E49E759400F515
:100D2B0095A10BC3E53394015002819A3064028183
:100D3B009AD802A14281C1C26DC2AF53E67F7591B1
:100D4B0000855394855495759104854D92854E93EA
:100D5B00D26043E680D2AFE52D54066008206A02CC
:100D6B000533020D80306D0D206C0A206407158150
:100D7B00158102161B2278003064027801E5377565
:100D8B00F007A4F9E5F028F5F0E9A2F013A2F113AE
:100D9B00A2F213F537C394785003753778C3E53750
:100DAB0095384008D265C295C294C293306002A1B7
:100DBB00B7854F92855093D26043E68022207D16F3
:100DCB00C2AF754202D291C292306202D293D2AFBD
:100DDB00759F11020FB7C2AF754202D291C290300C
:100DEB006202D295D2AF759F11020FB730724320BA
:100DFB007D20C2AF754203900135757B02C293D241
:100E0B0090306204D294C115C291D2AF759F01028A
:100E1B000FB7C2AF754203900135757B02C295D2F5
:100E2B0092306204D294C135C291D2AF759F210228
:100E3B000FB7207D17C2AF754203900110C29330DC
:100E4B006202D294D2AF759F01020FB7C2AF754247
:100E5B0003900110C295306202D294D2AF759F21DC
:100E6B00020FB7207D16C2AF754204D292C29030EA
:100E7B006202D294D2AF759F21020FB7C2AF7542F7
:100E8B0004D290C292306202D294D2AF759F01020B
:100E9B000FB7307243207D20C2AF754205900124FD
:100EAB00757B04C294D291306204D295C1BBC292BD
:100EBB00D2AF759F11020FB7C2AF754205900146B5
:100ECB00757B01C294D291306204D293C1DBC29084
:100EDB00D2AF759F11020FB7207D17C2AF754205B8
:100EEB00900106C294306202D295D2AF759F110267
:100EFB000FB7C2AF75420590011AC2943062EBD2A4
:100F0B0093D2AF759F11020FB7207D16C2AF7542FA
:100F1B0006D290C291306202D295D2AF759F010278
:100F2B000FB7C2AF754206D292C291306202D29312
:100F3B00D2AF759F21020FB7307243207D20C2AF15
:100F4B00754201900146757B01C295D292306204C5
:100F5B00D293E161C290D2AF759F21020FB7C2AF9E
:100F6B00754201900124757B04C293D290306204C8
:100F7B00D295E181C292D2AF759F01020FB7207D4E
:100F8B0017C2AF75420190011AC295306202D2931B
:100F9B00D2AF759F21020FB7C2AF75420190010608
:100FAB00C293306202D295D2AF759F01C265229077
:100FBB000104757B00C295C294C293D292D291D296
:100FCB0090C2622278807607087607087601087649
:100FDB00040876FF0876FF08760A08760208760181
:100FEB00087601788C76010876000876B40876FFCF
:100FFB000876FF0876FF0876030876FF0876010867
:10100B0076FF0876250876D00876780876C80876B5
:10101B00040876FF08760108760008767A08760AC7
:10102B000876010876010876000876FF087600221C
:10103B007887E6FFC2727888C27DE630E102D27D06
:10104B00C27E7889E630E102D27EC3EF940260085B
:10105B00758E01D273021068758E00C27322788070
:0D106B00E6149000809378A5F67881E614D5
:101078009000809378A6F67886E61490008D937891
:10108800A7F6789FE6F87005756B0001AFC3E89482
:101098001140027811E82828F56B256B256B28F597
:1010A8006C256B2828F56D7886E6F539C3940250CF
:1010B80003753902789CE67538FFB402037538A0C9
:1010C800B4030375388278A3E61490009A93F56602
:1010D800120FBA22227896E6FA7897E6FB7888E625
:1010E800B40305C3EB940EFB307F047A007BFFC387
:1010F800EB9AFCC3948250027C827572000572ECF4
:101108008572F0A4C3E5F0947D40F222D27F11DD10
:101118001205501205507A007B007C10120546E536
:101128005C2AFA74003BFBDCF37C04C3EB13FBEA98
:1011380013FADCF7FEC27F11DD22757C00757D0095
:10114800E5EF20E6037520000520903FFFE5201419
:101158006006901DFF1460009304600375EF16533A
:10116800D9BF7581C043FF8012054175EF0643B2B0
:1011780003E5B3240220E70DF521E5E320E0068529
:1011880021B343E301120FBA7580FF75A40075F10E
:101198009075D47F75908775A5BF75F2BF75D5001A
:1011A80075A60175E241120FBAE4F8F6D8FD756824
:1011B80001120FCF12167278988673753001C2AF7C
:1011C80012055A12056A12055012057112055012BD
:1011D800057812055012179912055A12055A120568
:1011E80055C2AF757C00757D0078FA79FA308707AB
:1011F800D9FBD8F7021C00113B116911DC11DD780D
:10120800988673120FBA75881075890275C8247587
:10121800910475D84075A82275B80275E690759B3B
:1012280080759D0075D10E75BC5875BB0675BA11D1
:1012380075E880120541D2AF12089975360053DA65
:10124800CF207E0343DA20307E0343DA1043DA01ED
:10125800C2D8C27112055AD2617B037A0CE55B7061
:10126800077A0CDB030211E9120550207003021102
:10127800E9C270E55CC3940240E1E52F541F855E26
:101288005DF55EB55DD5DAD5C26153DACF207E0350
:1012980043DA20307E0343DA10C2D8C27178A2E65E
:1012A8007008D274E52F54E0F52FC2757529001225
:1012B8000555307409C3E529940A4002D275120510
:1012C8004678023074027800C3E55C9840F0C2AFFB
:1012D80012056A12056A12056AD2AF12055A754CD0
:1012E80000120546788CE6C3940150030213D6E534
:1012F80030C3940150030213D6757CA5757DF12087
:101308007435C3E55C94FF50030213D6C2AF1205CF
:101318007FD2AF120555C3E55C940150EFC2AF12FE
:10132800056A12054B12056AD2AF120555C3E55C72
:1013380094FF40E902181E7F05D27F11DD12055582
:10134800C2AFC27F11DDAE5CC3E55C947FD2AF5003
:101358000261E6120541C2AF12057FD2AFDFDA3172
:1013680014C3EE94057897F612055A1217A17F0A4E
:10137800D27F11DD120555C2AFC27F11DDAE5CC34D
:10138800E55C947FD2AF50E6120541C2AF12056A00
:1013980012054B12056AD2AFDFD63114EE2403785A
:1013A80096F6F87997E7C394824003985006E824A4
:1013B800827897F612055A1216B41217D0120555EC
:1013C80011DDC3E55C94FF5002610102181E757CB3
:1013D80000757D00C3E55C954C4003855C4C1205A7
:1013E8005578017988E7B403027805C3E55C98402D
:1013F8000241E9C2AF12057F12057F12057FD2AF05
:1014080012055A753000E4F531F5320531E531F44D
:10141800703F0532789AE6781914601278321460B1
:101428000D787D14600878FA146003753200C3E5FE
:101438003298401D120FBA120541153275310078E5
:10144800998673C2AF12057FD2AF7898867312055A
:101458005512054BE52A700530740221E978012000
:0F14680074027806C3E55C9840A1120555E52A89
:1014770070030211E9C2AF120FBAE4F522F523F5A2
:1014870024F525F526F567D2AF7885E6C333F565EC
:10149700E4F544F545F546F547F548F570F52CF5BF
:1014A7002DF53775700875BB1012054112092A30E2
:1014B700EDFDA8BDA9BEE97001F8887112092E7566
:1014C700700875BB10113BC2AF7561FF1209E78544
:1014D7002261852262852263D2AF752201752401BC
:1014E700752501752601856069756A017888E6B4F6
:1014F7000307C27D307602D27DD268D26975330088
:10150700120F14120F43120A07120A0E120A0712B9
:101517000A0E120A07120C8C120660120D81120DA8
:10152700C8120A0E120C7B306E03120700206603E6
:10153700120853306603120883120D81120DF71239
:101547000A0E120C8C306E0312073C120D81120E1C
:101557006E120A0E120C7B306E0312079A120D815F
:10156700120E9D120A0E120C8C306E031207F71220
:101577000D81120F14120A0E12092A120C7B120D7A
:1015870081120F4312092E120A0E30692C856461ED
:10159700856462856069756A0179187A0CC3E533D9
:1015A700994009C269D26A8A350215C0C3E55C94BD
:1015B70001400302151C021623306A1D206C1AE530
:1015C70035147006C26AD26BA11CF535C3E55C946D
:1015D70001400302151C021623753600C3E55F940C
:1015E700014009856462856069756A0178FA79A4A2
:1015F700E760027803C3E55F985021307404E52A59
:10160700601A78F0306C058564617820C3E54198ED
:101617005002A11C0536E55C6002C126753600C282
:10162700AF120FBA7887E6FE7602113B7887EEF69F
:10163700E4F522F523F524F525F526F565752C0047
:10164700752D00D2AF120555120FBA78A4E66006C1
:10165700C292C291C290307406E52A700221E978DD
:101667008DE6C39401400241C6810E901A0D782081
:101677001216F6E520B4A50CA31216F6E520B45A07
:1016870003021694120FCF1216B40216B3901A0360
:1016970078807B0A1216F6A308DBF9901A0F788C6C
:1016A7007B191216F6A308DBF9901A2822C2AF128B
:1016B7001739121716901A00740E1216FBA3740727
:1016C7001216FBA374151216FB901A0378807B0A77
:1016D7001216FAA308DBF9901A0F788C7B191216E9
:1016E700FAA308DBF912174C12172A901A2822E4DA
:1016F70093F622E6438F01538FFDFFC3E583941CC6
:10170700400122EF857CB7857DB7F0538FFE2243DA
:101717008F02438F01857CB7857DB7901A0DF053F3
:101727008FFC22901A0D74A5D1FB901A0E745AD112
:10173700FB227A3079D07820901A40D1F6E520F74D
:1017470009A3DAF7227A3079D0901A40E7D1FB095A
:10175700A3DAF922AB74A875BB01027980BB020238
:101767007981BB03027982BB04027994BB050279B4
:1017770083BB06027986BB07027992BB0802798789
:10178700BB0902799CBB0A027988BB0B027989E8FD
:10179700F7227C0512055ADCFB22C2AF12056A123A
:1017A700057112057812057F12054B12056A12059D
:1017B7007112057812057F12054B12056A12057121
:1017C70012057812057FD2AF22C2AF12057F12052C
:1017D7007812057112056A12054B12057F120578FA
:1017E70012057112056A12054B12057F1205781250
:1017F700057112056AD2AF22AE74AF75C2AF12057A
:101807006A12056A12056A12054BDEF212057F128B
:10181700054BDFF8D2AF221217A1121799121799A9
:101827007574017575017576001217FF7C05AD5C3F
:1018370012055AC3ED955C70F5C3E55C9401400A47
:10184700C3E55C94FF403702186212175B1216B4A7
:101857001217A1C2AF75EF16121799DCD10576C31F
:0F186700E5769403500280C11217990575E57458
:101876001490009F93F808C3E57598500280A8124B
:1018860017991217990574C3E574940C5002809445
:0E189600120FCF1216B4C2AF75EF16121799CB
:0319FD0002114292
:101A00000E071507070104FFFF0A020101A55A018D
:101A100000B4FFFFFF03FF01FF25D078C804FF01DA
:091A200000FF0A010100FF00FFB4
:101A400023585031384123202020202020202020DE
:101A500023424C48454C4923463333302320202031
:101A60002020202020202020202020202020202076
:101C0000C2AFC2D353D9BF7581C043B20343FF8073
:101C1000752438752503B1DC7529A5752AF175E29F
:101C20004043F18053A47F75D4FFD2877DFA7803B7
:101C300079E67C10752200752300901DE97B0675FE
:101C400024987525013087028145208708D8FBD963
:101C5000F9DCF781B7308708D8FBD9F9DCF781B711
:101C6000B19CE493A3C39A6004DDC381B7DBDBB10D
:101C70008E6002812E7B08E493FAA3B16FDBF87AC1
:101C800030B16F752200752300B18EEAFCEBFDC305
:101C9000ED94FE400EB18E8A278B28ED30E0048A49
:101CA000828B83B18E7AC270D8C3ED94FE601950D6
:101CB000CEBD002BEC600F7520007521FF7529004B
:101CC000752A000200008100A827A9280809D80465
:101CD000D90281DCB192EA89AAF281CE0D81A3C337
:101CE000ED94035053EDA2E092007AC5C3E58294CF
:101CF00000E583941C508A200010438F02438F011B
:101D00008529B7852AB7F0300029A827A92808090E
:101D1000438F01538FFDD804D902A133C3E58394C7
:101D20001C4003A3A11689AAE28529B7852AB7F02A
:101D3000A3A116538FFC817F7AC1BD030CE493A34A
:101D4000FAB153DCF8B14B817F8181AA22AB23B178
:101D50006FEBFAEA6222752608C3E52313F523E543
:101D60002213F52250066323A0632201D526EAB18F
:101D7000DCB1DC75260AEAF4200102D287300102C8
:101D8000C287B1DCC3134002C201D526EB22B19257
:101D9000EAFB208702A192308702A197752608AE40
:101DA00024AF25C3EF13FFEE13FEB1E0B1DCC3EAAD
:101DB000133087024480FA30E703632201C3E5232E
:101DC00013F523E52213F52250066323A0632201B5
:101DD000D526D9E52265236523F52222AE24AF2539
:101DE0000E0FDEFEDFFCD20122424C48656C6934E6
:071DF000373163F3300601F7
:00000001FF
